:1000000009C016C015C014C013C012C011C010C062
:100010000FC00EC011241FBECFE9CDBF10E0A0E677
:10002000B0E001C01D92A236B107E1F726D054C05E
:10003000E7CF81E087BB83E088BB089590E020EEA6
:1000400031E087FF02C0C09A01C0C098F901319722
:10005000F1F79F5F983011F0880FF3CF089580E09B
:1000600090E020EE31E0880FB1998160F90131977D
:10007000F1F79F5F9830B9F708950F931F93CF93CF
:10008000DF9300EF10E010926100109260001BC03F
:10009000C0E0D0E082EBD2DF80916000CFDF21961C
:1000A000C035D105B9F78CEA9DE0F8013197F1F739
:1000B0000197D9F78091600090916100019690932B
:1000C00061008093600080916000909161008F3F9B
:0C00D000910509F0C4F6DCCFF894FFCFD6
:00000001FF
